:100000001CC036C136C069C033C032C01AC130C04E
:100010002FC02EC02DC02CC02BC02AC029C028C084
:1000200027C026C025C082C084C087C08AC08DC0BA
:1000300090C093C096C099C075C011241FBECFE573
:10004000D4E0DEBFCDBF11E0A0E6B0E0EEE5FCE01D
:1000500002C005900D92AC36B107D9F711E0ACE6BD
:10006000B1E001C01D92A538B107E1F79BD0F5C5FD
:10007000C7CF1F920F920FB60F9211248F93EF9359
:10008000FF9380916D018823B1F0E0916C01E9301C
:10009000D9F0959AF0E0E05AFF4F808183BD14BCFF
:1000A00085B5876085BDFF91EF918F910F900FBE51
:1000B0000F901F901895959AFF91EF918F910F9047
:1000C0000FBE0F901F9018959598FF91EF918F910B
:1000D0000F900FBE0F901F9018951F920F920FB6A2
:1000E0000F9211248F93959885B5887F85BD8F9148
:1000F0000F900FBE0F901F90189520E040E050E049
:10010000CA010197F1F72F5F2436D1F708958A309D
:1001100028F4E82FF0E0EA30F10508F00895ED5EEC
:10012000FF4F099480E185BBC198089515BAC19A23
:10013000089589E385BBC19A089584E285BBC1987F
:10014000089580E385BBC198089589E185BBC19876
:10015000089582E185BBC198089582E085BBC1986E
:10016000089588E385BBC19A089515BAC19808958A
:100170008F9A979A84B38F6384BBB99A80E090E09A
:10018000C6DF39D085B78C6085BF8BB780688BBFE1
:100190008D9A959A85B5886085BD89B7806889BF35
:1001A00078940895E5DF0EC08630C1F0853539F4C6
:1001B00080916D018823D1F0979A10926D01809102
:1001C0006C01A5DF81E01AD2823171F780916C0158
:1001D0008930A8F78F5F80936C01F1CF80916C011B
:1001E000882369F3815080936C01E9CF979881E06F
:1001F00080936D01E4CF10927201109273011092FE
:100200007401109275011092840110928301109272
:1002100076011092700110926E018EB589608EBDCC
:1002200089B7806189BF80EA90E09BBD8ABD85B7B0
:10023000826085BF8BB780648BBF8FB780688FBFAC
:1002400008951F920F920FB60F9211248F939F93D0
:10025000809180019091810101969093810180931A
:1002600080019F918F910F900FBE0F901F90189556
:100270001F920F920FB60F921124DF92EF92FF920E
:100280000F931F932F933F934F935F936F937F939E
:100290008F939F93AF93BF93CF93DF93EF93FF938E
:1002A0008BB78F7B8BBF7894809183019091840171
:1002B000892BE1F4C0918001D091810110928101DC
:1002C0001092800112BED090760181E0D81609F418
:1002D00045C0D81618F183E0D81609F4EFC084E0C1
:1002E000D81609F4A8C08BB780648BBFFF91EF913B
:1002F000DF91CF91BF91AF919F918F917F916F913E
:100300005F914F913F912F911F910F91FF90EF902F
:10031000DF900F900FBE0F901F9018958091700185
:10032000882309F416C1BE0180E090E0F5D17B017D
:100330008C0120E030E84AE454E498D118160CF01F
:1003400067C0C801B70120E030E847E754E4B9D1FD
:1003500087FF5EC081E08093760164C0BE0180E0CB
:1003600090E0DAD17B018C0120E030E84AEC53E4E4
:100370007DD11816B4F4C801B70120E030E847EF8A
:1003800053E49FD188236CF483E08093760110922C
:10039000710110926F0185B7836085BFD0927001A3
:1003A000A2CFC95CD040AC9798F580916E018823AC
:1003B00009F4D6C080916B00873009F4DFC08091CA
:1003C0006B0020916A00992787FD9095019633274D
:1003D00027FD30958217930709F4D5C080916B00F3
:1003E000873009F4EFC080916B008F5F80936B00C2
:1003F000E0916B00FF27E7FDF09580917701E858C9
:10040000FE4F808380916A008F3F11F410926A0042
:100410001092720110927301109274011092750182
:100420001092760185B78C7F85BF85B7826085BFC6
:100430001092700158CF80917001882309F453CF36
:1004400090917401809175018095981709F04BCFB8
:1004500080916B00873009F4A3C080916B002091DC
:100460006A00992787FD90950196332727FD3095DF
:100470008217930709F499C080916B00873009F4C3
:10048000A7C080916B008F5F80936B00E0916B0041
:10049000FF27E7FDF09580917401E858FE4F8083B7
:1004A000809174018093770180916A008F3F09F4F5
:1004B0008CC010926E0110928201AACF80917001BF
:1004C000882329F0E397629708F0A2CFABCFCE0143
:1004D0008A97409740F1BE0180E090E01DD17B01FA
:1004E0008C012AE939E148E153E4C0D018160CF038
:1004F0008FCFC801B70126E636EE49E353E4E1D0D9
:1005000087FF86CFE0916F01F0E0EE58FE4F20812B
:100510003091710181E090E002C0880F991F3A95F7
:10052000E2F7282B2083809171018F5F8093710106
:1005300080917101883069F41092710180916F018E
:100540008F5F80936F0180916F01843011F48093ED
:10055000760185B7836085BF81E080937001C3CE4B
:10056000809182018F5F809382018091820184302B
:1005700009F04ECF81E080936E014ACF80916A00EE
:10058000882309F01CCF80916A008F5F80936A00F6
:1005900080916A00883009F021CF10926A001ECF46
:1005A00080916A00882309F058CF80916A008F5F9C
:1005B00080936A0080916A00883009F05DCF1092C4
:1005C0006A005ACF10926B0013CF10926A0071CF5D
:1005D00010926B005BCF1092720110927301109217
:1005E0007401109275011092760185B78C7F85BFDA
:1005F00085B7826085BF1092700108958823E9F461
:1006000080916A008F3F59F1E0916A00FF27E7FD72
:10061000F095E858FE4FE08190916A0080916B0060
:100620009817A1F080916A008730E1F080916A000C
:100630008F5F80936A008E2F089580916A008F3FAC
:1006400019F780916A008F3FC1F3DECF8FEF80935F
:100650006B0080916B0080936A008E2F0895EFEFFE
:100660008E2F089510926A008E2F0895A8E1B0E0B1
:10067000EBE3F3E0C7C269837A838B839C832D838A
:100680003E834F83588789E0E82EF12CEC0EFD1E47
:10069000CE010196B701D9D18E010F5E1F4FCE0159
:1006A0000596B801D2D18985823038F089898230A7
:1006B00020F0C701B80141D201C08FEF6896E6E093
:1006C000BDC2A8E1B0E0E6E6F3E09CC269837A83AC
:1006D0008B839C832D833E834F83588789E0E82E4C
:1006E000F12CEC0EFD1ECE010196B701AED18E01AC
:1006F0000F5E1F4FCE010596B801A7D189858230C4
:1007000038F08989823020F0C701B80116D201C0C3
:1007100081E06896E6E092C2A8E0B0E0E1E9F3E0AB
:100720006DC27B018C01611571058105910519F47C
:1007300082E089835FC083E089838EE1C82ED12C5B
:10074000DC82CB82ED82FE820F831887C801B7015D
:1007500058D0FC013197F7FF3BC0222733272E1BCF
:100760003F0B57016801022E04C0D694C794B7947A
:10077000A7940A94D2F740E050E060E070E081E096
:1007800090E0A0E0B0E004C0880F991FAA1FBB1F33
:100790002A95D2F70197A109B1098E219F21A023A3
:1007A000B1230097A105B10521F041E050E060E0E0
:1007B00070E04A295B296C297D294D835E836F8314
:1007C00078878EE190E08E1B9F0B9C838B8312C0F9
:1007D000309781F00E2E04C0EE0CFF1C001F111F7D
:1007E0000A94D2F7ED82FE820F831887CE1ADF0AB1
:1007F000DC82CB821A82CE01019652D02896EAE0A2
:1008000019C2EF92FF920F931F937B018C0180E03E
:10081000E81680E0F80681E0080780E0180788F411
:100820008FEFE816F1040105110531F028F088E09A
:1008300090E0A0E0B0E017C080E090E0A0E0B0E081
:1008400012C080E0E81680E0F80680E0080781E04A
:10085000180728F088E190E0A0E0B0E004C080E153
:1008600090E0A0E0B0E020E230E040E050E0281B63
:10087000390B4A0B5B0B04C016950795F794E79468
:100880008A95D2F7F701E459FF4F8081281B31097F
:1008900041095109C9011F910F91FF90EF900895EF
:1008A000DF92EF92FF920F931F93FC01E480F5809B
:1008B00006811781D1808081823048F480E090E009
:1008C000A0E1B0E0E82AF92A0A2B1B2BA5C084304E
:1008D00009F49FC0823021F4EE24FF24870105C073
:1008E000E114F1040105110519F4E0E0F0E096C00F
:1008F000628173819FEF623879070CF05BC022E858
:100900003FEF261B370B2A3131052CF020E030E079
:1009100040E050E02AC0B801A701022E04C076953D
:100920006795579547950A94D2F781E090E0A0E04B
:10093000B0E004C0880F991FAA1FBB1F2A95D2F7E9
:100940000197A109B1098E219F21A023B12300970E
:10095000A105B10521F081E090E0A0E0B0E09A01AE
:10096000AB01282B392B4A2B5B2BDA01C9018F777E
:100970009070A070B07080349105A105B10539F474
:1009800027FF09C0205C3F4F4F4F5F4F04C0215CE1
:100990003F4F4F4F5F4FE0E0F0E02030A0E03A07DC
:1009A000A0E04A07A0E45A0710F0E1E0F0E0790186
:1009B0008A0127C06038710564F5FB01E158FF4FDB
:1009C000D801C7018F779070A070B0708034910506
:1009D000A105B10539F4E7FE0DC080E490E0A0E088
:1009E000B0E004C08FE390E0A0E0B0E0E80EF91EB4
:1009F0000A1F1B1F17FF05C016950795F794E7946C
:100A0000319687E016950795F794E7948A95D1F784
:100A100005C0EE24FF248701EFEFF0E06E2F67950D
:100A200066276795902F9F77D794DD24D7948E2FD4
:100A30008695492F462B582F5D29B701CA011F9172
:100A40000F91FF90EF90DF900895FC01DB01408152
:100A500051812281622F6F7770E0221F2227221F8F
:100A60009381892F880F822B282F30E0991F992797
:100A7000991F11969C93119721153105A9F54115E0
:100A800051056105710511F482E037C082E89FEFDE
:100A900013969C938E9312979A01AB0167E0220FF5
:100AA000331F441F551F6A95D1F783E08C930DC007
:100AB000220F331F441F551F12968D919C9113973F
:100AC000019713969C938E931297203080E03807FD
:100AD00080E0480780E4580758F314962D933D931F
:100AE0004D935C93179708952F3F310579F4411585
:100AF00051056105710519F484E08C93089564FF34
:100B000003C081E08C9312C01C9210C02F5730405C
:100B100013963C932E93129783E08C9387E0440FB7
:100B2000551F661F771F8A95D1F7706414964D93F1
:100B30005D936D937C93179708951F93DC01FB01E0
:100B40009C91923008F447C08081823008F443C001
:100B5000943051F411961C91843099F58181682F5D
:100B600070E0611B71093FC0843021F0923031F494
:100B70008230B9F18181882389F12DC011961C91B1
:100B800011978230F1F081811817D9F412962D91C6
:100B90003C911397828193818217930794F02817D1
:100BA0003907BCF014968D919D910D90BC91A02DAC
:100BB0002481358146815781281739074A075B0709
:100BC00018F4112341F00AC082179307A407B50750
:100BD00040F4112319F061E070E005C06FEF7FEF82
:100BE00002C060E070E0CB011F9108952F923F9208
:100BF0004F925F926F927F928F929F92AF92BF922D
:100C0000CF92DF92EF92FF920F931F93CF93DF93D8
:100C1000CDB7DEB7CA1BDB0B0FB6F894DEBF0FBE35
:100C2000CDBF09942A88398848885F846E847D8482
:100C30008C849B84AA84B984C884DF80EE80FD8084
:100C40000C811B81AA81B981CE0FD11D0FB6F894FA
:0E0C5000DEBF0FBECDBFED010895F894FFCFBB
:100C5E008D7D6D5E4E3E2F1F1001FFFF00010202C3
:100C6E000303030304040404040404040505050536
:100C7E000505050505050505050505050606060612
:100C8E0006060606060606060606060606060606F6
:100C9E0006060606060606060606060607070707E2
:100CAE0007070707070707070707070707070707C6
:100CBE0007070707070707070707070707070707B6
:100CCE0007070707070707070707070707070707A6
:100CDE000707070707070707070707070808080892
:100CEE000808080808080808080808080808080876
:100CFE000808080808080808080808080808080866
:100D0E000808080808080808080808080808080855
:100D1E000808080808080808080808080808080845
:100D2E000808080808080808080808080808080835
:100D3E000808080808080808080808080808080825
:100D4E000808080808080808080808080808080815
:0C0D5E0008080808080808080808080829
:00000001FF
